:030000000219FDE5
:03000B000200AA46
:03002B0002015D72
:03005B000202ECB2
:030073000202D9AD
:1000800002030406080C10182030406080040608A3
:100090000C10182030406080A0C00003070F1F0D17
:1000A0000D0403060D0503030202C2AFC0D0C0E079
:1000B000206214E5256009E473E525F4F58AD2622F
:1000C000D0E0D0D0D2AF3285268AC262E526F46075
:1000D0003030682620720DD0E0D0D0C290C291C2DC
:1000E00092D2AF32C290C291C292206F0D20660AA6
:1000F0007401D5E0FDE57BF45290D0E0D0D0D2AFD2
:1001000032758A00C28DD26201FA01B930680520C9
:100110006602D29001B9306805206602D29101B919
:10012000306805206602D29201B9D29330680A2065
:1001300066077405D5E0FDD29001B9D29430680A03
:100140002066077405D5E0FDD29101B9D2953068DB
:100150000A2066077405D5E0FDD29201B9C2AFC28C
:10016000AD53E6EFC0D0C0E0D2D3D2AFC2CEE52AC5
:100170006007207449152A21BE7800790020742E6A
:10018000E580307E01F430E70278FF53DACF207E3D
:100190000343DA20307E0343DA10C2D8C271E5800F
:1001A000307E01F430E70279FFC3E89970CB30610B
:1001B00003752A40207403752A40885CD27020742D
:1001C0000DE52B6004152B21CE43DA01C2D8207037
:1001D0000221E1A85C206102C27020740221DF8844
:1001E000227882B60403852224C3E5259440400288
:1001F000D26420CF0AD0E0D0D043E610D2AD32C2D4
:10020000CF053A7802E52A6005307402152AC3E565
:100210005C94014005755F00412B756000756900B5
:10022000E55F2401F55F5003755FFF7982B7020D2A
:10023000306E1DC3E52294324016854C227982B778
:10024000030E306E0BC3E52294324004798E872270
:10025000C3E5239522600840041523415F0523D898
:10026000CA0569E56970021569D56A63756A01781E
:1002700005C3E569956B4057C3E569956C500878EF
:1002800001756A03020293C3E569956D5005780113
:10029000756A01C3E5629524401E7982B704024164
:1002A000C4206E14852462E569046003856B69755A
:1002B0006A0175233C0202CFE5622850057562FF92
:1002C00041C4F562E5620470067560FF7569FFD090
:1002D000E0D0D043E610D2AD32C2AF53E67F759284
:1002E000FA7593FFC260759104D2AF32C2AF53E684
:1002F000EFC2ADC0D0C0E0C0F0D2D3D2AFA8FBA94E
:10030000FCC2D8307102615353DACF207E0343DA46
:1003100010307E0343DA20D271E580307E01F42074
:10032000E702612A88278928A13853DACF207E0383
:1003300043DA20307E0343DA10C2D8C2713074022F
:10034000A1247800E580307E01F430E702A1248802
:100350005CA10C53DACF207E0343DA20307E0343C6
:10036000DA10C271206102812C53DACF207E034360
:10037000DA10307E0343DA20C2D8D2718857895808
:10038000C3E89555F8E99556F97B007E087A00C3D5
:10039000E8948CE994005005755B00811E882178F3
:1003A000A2E6A8216055C3E894C8E994005008E487
:1003B000D2E4FB7A0A61F9C3E89468E99401500831
:1003C000E4D2E3FB7A0F61F9C3E894D0E9940250D8
:1003D00008E4D2E2FB7A1E61F9C3E894A0E994052F
:1003E0005008E4D2E1FB7A3C61F9C3E89498E994BF
:1003F000085008E4D2E0FB7A787E00C3E89559FC07
:10040000E9955AFD30E70AECF42401FCEDF43400E0
:10041000FD755B00C3EC9AED9E5003755B01885936
:10042000895A8557558558567802A10CC3E89527F7
:10043000F8E99528F9307C0281F0307B0281F030B8
:100440007A0281E9207502814FE9FDE8FC816EE9BD
:10045000C313F9E813F830790281E9E9C313F9E825
:1004600013F830780281E9E9C313FDE813FC206139
:0F0470002CC3EC941CED940240028185ED701EAC
:10047F00C3EC94C850180529E52970021529C3E566
:10048F0029940A5002A124755C00D270A124E52999
:10049F00600215297400207F037896E624FAFEE4A3
:1004AF003400FFC3EC9EFCED9FFD500678007900F1
:1004BF0081F0C3EC94FFED9400400678FF79008142
:1004CF00F0EC8572F0A4C5F0A2F733F87900400381
:1004DF0002050C78FF790002050CE9C313F9E81344
:1004EF00F8307C0EE9600278FFC3E81338F8E43483
:1004FF0000F9C3E894FFE99400400278FF885CD2CA
:10050F0070206102A124741FF4552F4BF52FC27474
:10051F00EB7002D274752A40307403752A0A306169
:10052F0002A13820740353DAFE207403752B20D0F8
:10053F00F0D0E0D0D0D2AD43E61032790102056899
:10054F007903020568790A020568791E0205687940
:10055F006402056879C80205687817E4D5E0FDD80C
:10056F00FAD9F6227A147B7802058F7A107B8C02E7
:10057F00058F7A0D7BB402058F7A0B7BC802058F2E
:10058F007902E4D294D5E0FDD291D5E0FDC291D5A8
:10059F00E0FDC294D5E0FDE920E002D29030E00208
:1005AF00D292E573D5E0FDE920E002C29030E0027F
:1005BF00C2927496D5E0FDD9C9EAF8D5E0FDD8FB13
:1005CF00DBBED29422C37C007D0075F00005F0EAFB
:1005DF0033FAEB33FB50F6EB13FBEA13FAC3E9FFE5
:1005EF00E8FEE89AF8E99BF95004EFF9EEF8B3EC5E
:1005FF0033FCED33FDD5F0DFEDF9ECF822E889F0AF
:10060F008A20D2D4F8A9F07B0030F70B7BFFF424BB
:10061F0001F8E9F43400F9E88520F0A4ADF0F8E929
:10062F008520F0A4AFF0FEED2EF974003FFA7C04A4
:10063F00C3EA13FAE913F9E813F8DCF48BF030F797
:10064F000AE8F42401F8E9F43400F9E889F0C2D497
:10065F00F8A9F0227882B60403020702C3E55C947E
:10066F0019401EE52D54067018206E3678057994C2
:10067F00E7146007780A1460027812C3E5419840C6
:10068F001F306E098564627569FF756A01852224C2
:10069F00E4F544F545F546F547F548C26E02070205
:1006AF00D26E7994E7147013E523F43333F913F80A
:1006BF00E9540104F9E854FE0206F6E71414701425
:1006CF00E523F4333333F913F8E9540304F9E85409
:1006DF00FC0206FEE523F433333333F913F8E95400
:1006EF00070404F9E854F8C39440F8E99400F98832
:1006FF0044894522C3E54113F9E54013F8C3E544A6
:10070F0098F8E54599F9500CC3E89480E994FF40B7
:10071F001602073AC3E8947FE99400500302073AA0
:10072F00787F790002073A788079FF8849894A22D1
:10073F00E5492546F8E54A3547F9854A20E430076B
:10074F0001F43548FA30E709C3EA94F0401502077F
:10075F0078C3EA940F500302077878FF79FF7A0F76
:10076F00020778780079007AF0C3E5249561500A82
:10077F00C374019524500B020796E54A20E70E0239
:10078F000796E54A30E706884689478A482278A5C2
:10079F00E6FAC3E54933F8E54A33F9D10CE930E716
:1007AF000BC3E89480E994FF4013E1D0C3E8947F32
:1007BF00E994005002E1D0787F7900E1D078807918
:1007CF00FFE820E715C3E52398F84009C3E8940133
:1007DF0040030207F778010207F7E8F42401252305
:1007EF00F840030207F778FF884B2278A6E6FAA8AD
:1007FF0047A94812060CE930E70CC3E89401E994C5
:10080F00FF401602082CC3E894FFE994005003023E
:10081F00082C78FF790002082C780179FFE920E78E
:10082F0015C3E54B98F84009C3E89401400302084B
:10083F00537801020853E8F42401254BF8400302D2
:10084F00085378FF88242278FFC26420693D206A0C
:10085F0012D264C3E541940A4009C3E52594405080
:0E086F0002C26479A1E76023E541601F74FFB7
:10087D008541F0848539F0306A0375F005A4F8C51B
:10088D00F0600278FFC3E895645002A86488632283
:10089D00C3E5409440E5419401E56350031401AE76
:1008AD00046002F563227883E6F520120F2B75E8BC
:1008BD009012054A75E890E5E820ECFBA8BDA9BEAD
:1008CD00120FD1756EEC756F01C3740113FD74ECCD
:1008DD00606613FC74EC2CFC74013DFDECFAEDFB31
:1008ED00C3E89AE99B4014E56E24ECF56EE56F3490
:1008FD0001F56FEA2CFAEB3DFB80E5AE6EAF6FC3F1
:10090D00E56F13F9E56E13F8C3E913F9E813F87AF7
:10091D0003C3E913F9E813F8DAF7AA201A70097579
:10092D006E00756F000209451AEA6008EE28FEEFA9
:10093D0039FFDAF88E6E8F6F2275E890227883E694
:10094D00FFE5E820ECF7A8BDA9BE0570C3E57094DE
:10095D00084052757000E9FA79A0E76044EA700723
:10096D00E571601B020980C3E895716010E5715057
:10097D0006600C1402098C0460F902098CE571F50E
:10098D0071C394F6401B7561C0C394064013756125
:10099D0080C39406400B756140C394064003756196
:1009AD000075BB0622EFC39401601F74EC601BC37E
:1009BD00E894FFE994035012C3E8956EE9956F50E2
:1009CD0009E561600C15610209DEE561F46002055F
:1009DD0061A861C3E524985002A824C3E89562403C
:1009ED000AA862E562F4600385626188258826E5C0
:1009FD0070B4070375BB1022743279A787F0A4C5B4
:100A0D00F0A2F733F8C3E895614002A86188228807
:100A1D0024882588268864227540007541F022C2FD
:100A2D00AF75C820A8CCA9CDAA3A30CF010A75C898
:100A3D0024D2AFAB3BAC3C883B893CC3E89BF8E987
:100A4D009C206908F930670261384195AD3D8A3DBA
:100A5D00F9EA9DFA600478FF79FFAE3EAF3F8B3E19
:100A6D008C3FA83BA93CC3E89EF8E99FF9C3E5413B
:100A7D0013FBE54013FAE82AF540E93BF541500632
:100A8D007540FF7541FF41DFAA40AB41AC40AD4120
:100A9D007E047F02C3EB940440021E1FC3EB940837
:100AAD0040021E1FC3ED13FDEC13FCDEF7C3EA9CE1
:100ABD00FAEB9DFBEF6009C3E913F9E813F8DFF7D3
:100ACD00EA28FAEB39FB8A408B4150067BFF8B40BD
:100ADD008B41C3EB94025002D2673069047F0361EE
:100AED000A7892E6FFC3E537948240110FC3E537CC
:100AFD0094A040010FC3EF940640027F057E02E5EE
:100B0D0041C4540FF9E541C454F0F8E540C4540F05
:100B1D0028F8C3E89EFAE99400FB4009C3EA940261
:100B2D00EB940050047A02E4FB6184AA40AB41EBE4
:100B3D00C4FEEAC4540F4EFCC3EA9CFAEB9400FBCE
:100B4D00C3E813C313F8EA28FAEB3400FB8A408B91
:100B5D0041C3EB94024002C2677802EBC4FE7B00F6
:100B6D00EAC4540F4EFAC3EA98FA4005C3940250F2
:100B7D00027A027892E6FF30600261848551928597
:100B8D005293D26043E680C3E49AF8E49BF9306750
:100B9D00028110E8FAE9FBD3E913FDE813FC885153
:100BAD008952C3EF94036038EF20E00DE82CF8E98B
:100BBD003DF9ECFAEDFB020BD9E828F8E939F9C358
:100BCD00E82402F8E93400F97AFE7BFFC3EF9403C1
:100BDD00400E8A538B54884D894E8C4F8D508144D5
:100BED00885389548A4D8B4E8C4F8D5030691275B8
:100BFD0053F07554FF754FF07550FF7551F07552E8
:100C0D00FF8144E8FAD3E813FC8851C3EF940360E5
:100C1D0020EF20E007E82CF8ECFA8130E8282402D8
:100C2D00F87AFEC3EF940340088A53884D8C4F81A8
:100C3D004488538A4D8C4FE568C3335002646BF57D
:100C4D0068306002814E753402D26043E680E52D36
:100C5D0054066034A840A941C3E913F9E813F8C359
:0F0C6D00E913F9E813F8306904E92440F9C2AF3C
:100C7C0053E67F759100C3E498F594E499F5957566
:100C8C009104D26043E680D2AF22D26575430075E1
:100C9C002000306C03752040020CB5D26575430002
:100CAC00752040306C037520007801790120672095
:100CBC00E52D54066002C2657914E541C313700139
:100CCC0004F8C3941440027814306904781B791B1F
:100CDC00206010E543600C306903D53404D26DA15B
:100CEC005891560543E59BF45440B52002A142307F
:100CFC00690908C3E89940011881DC20650A08C31A
:100D0C00E899400281B581DCC265C2AF53E67F75BC
:100D1C0091003067127594007595FE759104D26040
:100D2C0043E680D2AF81B5AE40AF41C3E49EF594AB
:100D3C00E49FF595A127C3E5339401500281B530AA
:100D4C00650281B5D802A15681DCC26DC2AF53E6F3
:100D5C007F759100855394855495759104854D92BA
:100D6C00854E93D26043E680D2AFE52D54066008E1
:100D7C00206A020533020D94306D0D206C0A20653B
:100D8C00071581158102160922780030640530653B
:100D9C00027801E53775F007A4F9E5F028F5F0E9DC
:100DAC00A2F013A2F113A2F213F537C394785003F7
:100DBC00753778C3E53795384008D266C290C29132
:100DCC00C292306002A1CE854F92855093D260437F
:100DDC00E68022207D16C2AF754202D294C29330B7
:100DEC006202D292D2AF759F11020FCEC2AF754282
:100DFC0002D294C295306202D290D2AF759F11028A
:100E0C000FCE307243207D20C2AF75420390013B60
:100E1C00757B10C292D295306204D291C12CC294CF
:100E2C00D2AF759F01020FCEC2AF75420390013B4A
:100E3C00757B10C290D293306204D291C14CC29493
:100E4C00D2AF759F21020FCE207D17C2AF75420322
:100E5C00900116C292306202D291D2AF759F0102FC
:100E6C000FCEC2AF754203900116C290306202D20F
:100E7C0091D2AF759F21020FCE207D16C2AF754265
:100E8C0004D293C295306202D291D2AF759F2102E7
:100E9C000FCEC2AF754204D295C293306202D2918A
:100EAC00D2AF759F01020FCE307243207D20C2AFAE
:100EBC0075420590012A757B08C291D29430620468
:100ECC00D290C1D2C293D2AF759F11020FCEC2AFD6
:100EDC0075420590014C757B20C291D2943062040E
:100EEC00D292C1F2C295D2AF759F11020FCE207D66
:100EFC0017C2AF75420590010CC291306202D290BC
:100F0C00D2AF759F11020FCEC2AF75420590012072
:100F1C00C2913062EBD292D2AF759F11020FCE20EC
:100F2C007D16C2AF754206D295C294306202D29041
:100F3C00D2AF759F01020FCEC2AF754206D293C2DB
:100F4C0094306202D292D2AF759F21020FCE3072D2
:100F5C0043207D20C2AF75420190014C757B20C2AD
:100F6C0090D293306204D292E178C295D2AF759F41
:100F7C0021020FCEC2AF75420190012A757B08C2C7
:100F8C0092D295306204D290E198C293D2AF759F01
:100F9C0001020FCE207D17C2AF754201900120C215
:100FAC0090306202D292D2AF759F21020FCEC2AFA7
:100FBC0075420190010CC292306202D290D2AF7590
:100FCC009F01C2662290010A757B00C290C291C239
:100FDC0092D293D294D295C2622278807607087608
:100FEC00070876010876040876FF0876FF08760B6A
:100FFC00087602087601087601788C76010876006E
:10100C000876B40876FF0876FF0876FF08760308A2
:10101C0076FF0876010876FF0876250876D00876E4
:10102C00780876C80876040876FF087601087600FA
:10103C0008767A08760708760108760108760008A3
:10104C0076FF087600227887E6FFC272BF0302D2D1
:10105C00727888C27DE630E102D27DC27E7889E664
:0E106C0030E102D27EC3EF94026008758E015F
:10107A00D273021084758E00C273227880E61490AF
:10108A0000809378A5F67881E6149000809378A67C
:10109A00F67886E61490008D9378A7F6789FE6F89E
:1010AA00700108C3E8941140027811E82828F56B0A
:1010BA00256B256B28F56C256B2828F56D7886E657
:1010CA00F539C394025003753902789CE67538FFE6
:1010DA00B402037538A0B4030375388278A3E61402
:1010EA0090009A93F566120FD122227896E6FA7842
:1010FA0097E6FB7888E6B40305C3EB940EFB307FD2
:10110A00047A007BFFC3EB9AFCC3948250027C8270
:10111A007572000572EC8572F0A4C3E5F0947D4007
:10112A00F222D27F11F51205597A007B007C101247
:10113A00054FE55C2AFA74003BFBDCF37C04C3EB45
:10114A0013FBEA13FADCF7FEC27F11F522E5EF2062
:10115A00E6037520000520903FFFE5201460069005
:10116A001DFF1460009304600375EF1053D9BF7517
:10117A0081C043FF8012054A75EF0043B203E5B30D
:10118A00240220E70DF521E5E320E0068521B3439B
:10119A00E301120FD17580FF75A40075F19075D423
:1011AA007F75903875A53F75F23F75D50075A60114
:1011BA0075E241120FD1E4F8F6D8FD756801120FF5
:1011CA00E612166078988673753001C2AF1205630D
:1011DA0012057312055912057A1205591205811260
:1011EA00055912178312056312056312055EC2AF11
:1011FA0078FA79FA308707D9FBD8F7021C0011521E
:10120A00118511F411F578988673120FD17588102B
:10121A0075890275C82475910475D84075A8227518
:10122A00B80275E690759B80759D0075D10775BCEF
:10123A005875BB0675BA1175E88012054AD2AF1205
:10124A0008B375360053DACF207E0343DA20307EA6
:10125A000343DA1043DA01C2D8C271120563D261BC
:10126A007B037A0CE55B70077A0CDB030211F81238
:10127A0005592070030211F8C270E55CC39402405C
:10128A00E1E52F541F855E5DF55EB55DD5DAD5C201
:10129A006153DACF207E0343DA20307E0343DA102B
:1012AA00C2D8C27178A2E67008D274E52F54E0F56C
:1012BA002FC27575290012055E307409C3E5299499
:1012CA000A4002D27512054F78023074027800C3C0
:1012DA00E55C9840F0C2AF120573120573120573EC
:1012EA00D2AF120563754C0012054F788CE6C39491
:1012FA000150030213C8E530C3940150030213C816
:10130A00207435C3E55C94FF50030213C8C2AF12C0
:10131A000588D2AF12055EC3E55C940150EFC2AFF7
:10132A00120573120554120573D2AF12055EC3E596
:10133A005C94FF40E90218087F05D27F11F5120577
:10134A005EC2AFC27F11F5AE5CC3E55C947FD2AFDB
:10135A00407612054AC2AF120588D2AFDFDC312CC3
:10136A00C3EE94057897F61205631216A212178B2C
:10137A007F0AD27F11F512055EC2AFC27F11F5AEA8
:10138A005CC3E55C947FD2AF50E612054AC2AF1245
:10139A000573120554120573D2AFDFD6312CEE2431
:1013AA00037896F61205631216A21217BA12055E90
:1013BA0011F5C3E55C94FF5002610A021808C3E5FF
:1013CA005C954C4003855C4C12055E78017988E790
:1013DA00B403027805C3E55C98400241F2C2AF1239
:1013EA000588120588120588D2AF12056375300088
:1013FA00E4F531F5320531E531F4703F0532789A7A
:10140A00E67819146012783214600D787D14600839
:10141A0078FA146003753200C3E53298401D120F42
:10142A00D112054A153275310078998673C2AF1206
:10143A000588D2AF7898867312055E120554E52A9C
:10144A00700530740221F878012074027806C3E529
:10145A005C9840A112055EE52A70030211F8C2AF3A
:0E146A00120FD1E4F522F523F524F525F52621
:10147800F567D2AF7885E6C333F565E4F544F545FD
:10148800F546F547F548F570F52CF52DF5377570E7
:101498000875BB1012054A120946E5E820ECFBA8BE
:1014A800BDA9BEE97001F8887112094A75700875FE
:1014B800BB101152C2AF7561FF120A058522618502
:1014C8002262852263D2AF75220175240175250138
:1014D800752601856069756A017888E6B40307C2D4
:1014E8007D307602D27DD268D269753300120F2B17
:1014F800120F5A120A25120A2C120A25120A2C1245
:101508000A25120CA7120663120D95120DDF120A96
:101518002C120C96306E031207032067031208562C
:1015280030670312089D120D95120E0E120A2C1226
:101538000CA7306E0312073F120D95120E85120A82
:101548002C120C96306E0312079D120D95120EB4D4
:10155800120A2C120CA7306E031207FA120D9512FC
:101568000F2B120A2C120946120C96120D95120F07
:101578005A12094A120A2C30692C85646185646202
:10158800856069756A0179187A0CC3E53399400951
:10159800C269D26A8A350215AEC3E55C940140037C
:1015A80002150A021611306A1D206C1AE5351470EE
:1015B80006C26AD26BA10AF535C3E55C9401400303
:1015C80002150A021611753600C3E55F9401400939
:1015D800856462856069756A0178FA79A4E76002B2
:1015E8007803C3E55F985021307404E52A601A78BF
:1015F800F0306C058564617820C3E541985002A1FC
:101608000A0536E55C6002C114753600C2AF120FD8
:10161800D17887E6FE760211527887EEF6E4F52255
:10162800F523F524F525F526F565752C00752D00AF
:10163800D2AF12055E120FD178A4E66006D290D21E
:1016480091D292307406E52A700221F8788DE6C3AB
:101658009401400241CF61FA901A0D78201216E4E5
:10166800E520B4A50CA31216E4E520B45A0302162B
:1016780082120FE61216A20216A1901A0378807B36
:101688000A1216E4A308DBF9901A0F788C7B19125A
:1016980016E4A308DBF9901A2822C2AF1217231206
:1016A80016FD901A00740E1216E9A374061216E9B4
:1016B800A374151216E9901A0378807B0A1216E8AB
:1016C800A308DBF9901A0F788C7B191216E8A30887
:1016D800DBF9121736121714901A2822E493F6220F
:1016E800E6438F01538FFD75EF0275B7A575B7F106
:1016F800F0538FFE22438F02438F0175EF0275B7B7
:10170800A575B7F1901A0DF0538FFC22901A0D743D
:10171800A5D1E9901A0E745AD1E9227A3079D07895
:1017280020901A40D1E4E520F709A3DAF7227A30AD
:1017380079D0901A40E7D1E909A3DAF922AB74A865
:1017480075BB01027980BB02027981BB03027982F1
:10175800BB04027994BB05027983BB06027986BB78
:1017680007027992BB08027987BB0902799CBB0AF8
:10177800027988BB0B027989E8F7227C0512056398
:10178800DCFB22C2AF12057312057A12058112051D
:101798008812055412057312057A120581120588FC
:1017A80012055412057312057A120581120588D2A2
:1017B800AF22C2AF12058812058112057A1205738D
:1017C80012055412058812058112057A1205731242
:1017D800055412058812058112057A120573D2AFD5
:1017E80022AE74AF75C2AF1205731205731205737A
:1017F800120554DEF2120588120554DFF8D2AF2222
:1018080012178B121783121783757401757501757A
:1018180076001217E97C05AD5C120563C3ED955C93
:1018280070F5C3E55C9401400AC3E55C94FF40375A
:1018380002184C1217451216A212178BC2AF75EF79
:1018480010121783DCD10576C3E576940350028025
:10185800C11217830575E5741490009F93F808C3A7
:0F186800E57598500280A8121783121783057434
:10187700C3E574940C50028094120FE61216A2C2AC
:07188700AF75EF101217838B
:0319FD000211577D
:101A00000E061507070104FFFF0B020101A55A018D
:101A100000B4FFFFFF03FF01FF25D078C804FF01DA
:091A200000FF07010100FF00FFB7
:101A40002345415A5933417632232020202020203B
:101A500023424C48454C4923463333302320202031
:101A60002020202020202020202020202020202076
:101C0000C2AFC2D353D9BF7581C043B20343FF8073
:101C1000752438752503B1C975EF0275E24043F1AB
:101C20008053A47F75D4FFD2877DFA780379E67C50
:101C300010752200752300901DD67B0675249875BB
:101C400025013087028142208708D8FBD9F9DCF7CB
:101C500081B4308708D8FBD9F9DCF781B4B189E4C5
:101C600093A3C39A6004DDC381B4DBDBB17B600264
:101C7000812B7B08E493FAA3B15CDBF87A30B15C8A
:101C8000752200752300B17BEAFCEBFDC3ED94FEE9
:101C9000400EB17B8A278B28ED30E0048A828B834B
:101CA000B17B7AC270D8C3ED94FE601350CEBD00F4
:101CB00025EC60097520007521FF0200008100A855
:101CC00027A9280809D804D90281D3B17FEA89AAB3
:101CD000F281C50D81A0C3ED94035049EDA2E092BD
:101CE000007AC5C3E5829400E583941C50902000DF
:101CF00010438F02438F0175B7A575B7F1F030001F
:101D00001FA827A9280809438F01538FFDD804D99C
:101D100002A12089AAE275B7A575B7F1F0A3A10DBC
:101D2000538FFC817C7AC1BD030CE493A3FAB140CC
:101D3000DCF8B138817C817EAA22AB23B15CEBFA5E
:101D4000EA6222752608C3E52313F523E52213F57D
:101D50002250066323A0632201D526EAB1C9B1C986
:101D600075260AEAF4200102D287300102C287B147
:101D7000C9C3134002C201D526EB22B17FEAFB2082
:101D80008702A17F308702A184752608AE24AF2583
:101D9000C3EF13FFEE13FEB1CDB1C9C3EA13308711
:101DA000024480FA30E703632201C3E52313F523DD
:101DB000E52213F52250066323A0632201D526D91C
:101DC000E52265236523F52222AE24AF250E0FDE22
:101DD000FEDFFCD20122424C48656C693437316326
:041DE000F3300601D5
:00000001FF
